:100000009CC02AC2B6C0B5C0B4C0B3C0B2C0B1C0F3
:10001000B0C0AFC0AEC0ADC0ACC0ABC0AAC0A9C07C
:10002000A8C0040309045A03680061006600740054
:100030006D0061006E006E00230073006F006600AB
:1000400074007700610072006500200028007700CE
:10005000770077002E00740075002D0063006800A3
:1000600065006D006E00690074007A002E00640067
:1000700065002F007E0068006500680061002900AF
:100080003003480049004400200046006C0079001D
:1000900053007400690063006B00200028004A00D0
:1000A0006F00790073007400690063006B00290021
:1000B0003A03680065006800610040006800720053
:1000C0007A002E00740075002D0063006800650042
:1000D0006D006E00690074007A002E0064006500F7
:1000E0003A003000300031003000120110010000F1
:1000F0000008C016DB2700010102030109022200EB
:10010000010100800A090400000103000000092128
:1001100001010001221B00070581030800100501F1
:100120000904A101150025017501950205091901B0
:100130002902810295068101C00011241FBECFE56E
:10014000D1E0DEBFCDBF10E0A0E6B0E0EEE4F9E024
:1001500003C0C89531960D92A236B107D1F710E0D1
:10016000A2E6B0E001C01D92AE39B107E1F781D33C
:10017000EDC346CF8BB780648BBF8BE48093730055
:100180008AE58093720008950F931F93CF93DF93B6
:1001900010918400135017FDB6C00091800080912B
:1001A0007F008D3209F0ADC08AEF3CD380917F0093
:1001B0008D3209F0A6C0183009F0A3C0C4E9D0E020
:1001C000C01BD10983EC809367008AE580936000AF
:1001D000109262008881807621F08C2F9D2F31D380
:1001E00086C09A81109270008981882321F4109230
:1001F000710082E076C0853019F49093850070C05C
:10020000863009F059C08B81813041F48AEE90E04C
:10021000909383008093820092E149C0823041F440
:100220008CEF90E0909383008093820092E23FC035
:10023000833041F5992341F482E290E0909383006A
:100240008093820094E033C0913041F486E290E0E4
:1002500090938300809382009AE529C0923041F404
:1002600080E890E0909383008093820090E31FC029
:100270009330E1F480EB90E09093830080938200D0
:100280009AE315C0813241F48CE391E090938300AE
:100290008093820099E00BC0823241F48EE191E0BC
:1002A00090938300809382009BE101C090E080E402
:1002B00080936200892F1BC0883021F481E027E8F9
:1002C00030E011C0893019F49093870009C08A305A
:1002D00011F481E006C08B3019F48BE48093730035
:1002E00080E020E730E03093830020938200282FC5
:1002F0008F81882321F48E81821708F4282F209380
:100300006100109284008091600084FF4AC0609177
:1003100061006F3F09F445C090916700693008F0B3
:100320004BC01092610088E898279093670066237D
:1003300009F44BC0209182003091830080916200CB
:1003400086FF0CC0962FF32FE22FA8E6B0E0C895E9
:10035000802D8D9331969150D1F709C0962FF32FB0
:10036000E22FA8E6B0E081918D939150E1F76150C2
:10037000932F822F860F911D6F5F019690938300BC
:10038000809382007727162F88E690E061D01C5F6B
:100390001C3010F01CE003C08FEF809361001093BD
:1003A000600094E186B38670B1F49150D9F7109251
:1003B000850010927E000FC068506093610088E84D
:1003C00098279093670068E0B5CF60E088E690E0FA
:1003D0003FD014E0E1CFDF91CF911F910F910895AD
:1003E0001F93B92FA82F162F8091720084FF07C08A
:1003F0008091730098E889278093730003C08AE591
:1004000080937200912FE4E7F0E08D9181939150F9
:100410001916DCF3612F84E790E01AD01C5F10936B
:1004200072001F910895A82FB92F80E090E041E05D
:1004300050EA60956F5F58F42D9138EF82279795B9
:10044000879510F0842795273F5FC8F3F3CF089571
:10045000EADF8D939D930895CF93CFB7CF93C39544
:10046000B29BE9F7B29B1DC0B29B1BC0B29B19C0E7
:10047000B29B17C0B29B15C0C0918100C395C093B9
:100480008100DF93DD27C2B7D2BFC85CD1B7C230CD
:1004900012F0D15003C0CF3F0AF4D395D1BFDF9102
:1004A0003EC1DF93C0918000DD27C857DF4FB29B6C
:1004B00002C0DF91D7CF2F930F931F9320E8B299FB
:1004C00021604F933F930F92B29922601FEF3BE060
:1004D000022F220F00C0B2990C602027087046B38B
:1004E00011F4000036C0B4C042FFC89546B320687E
:1004F00000000227B29B0AC0287F11F046B388C0D3
:1005000046B31E7FB29BB19901C06AC042FDC89537
:1005100046B321604670B29908C0B9F3217F46B353
:1005200009F087C01D7F00C000C042FFC89546B3D8
:1005300022600000B29B08C0237E11F046B387C042
:1005400046B31B7F00C000C042FDC89546B324607F
:100550000993B29908C0277C11F046B387C046B30F
:10056000177F00C000C042FFC89546B32860012F26
:10057000B29B08C02F7811F046B387C046B30F7EF8
:1005800000C000C042FDC89546B320611FEFB2997C
:1005900008C02F7111F046B387C046B30F7D00C06D
:1005A00000C042FFC89546B32062315038F0B29B7C
:1005B00008C02F73223046B314F085C08EC00F7B65
:1005C000C89542FDC89546B320640000B2998CCF0F
:1005D0002F77243046B30CF00AC00F77000084CF89
:1005E00009937DC042FDC89546B3206800000227EC
:1005F000B2990AC0287F11F046B38CCF46B31E7F54
:10060000B29BB19901C0ECCF42FFC89546B32160BF
:100610004670B29B09C0217F19F046B300008ACF13
:1006200046B31D7F00C000C042FDC89546B3C1F26D
:100630002260B29908C0237E11F046B389CF46B339
:100640001B7F00C000C042FFC89546B324600993D9
:10065000B29B08C0277C11F046B389CF46B3177F01
:1006600000C000C042FDC89546B32860012FB29972
:1006700008C02F7811F046B389CF46B30F7E00C073
:1006800000C042FFC89546B320611FEFB29B08C06F
:100690002F7111F046B389CF46B30F7D00C000C063
:1006A00042FDC89546B320623150B8F0B29907C0F8
:1006B0002F73223046B30CF089CF0F7BC89542FFD1
:1006C000C89546B32064B29B8DCF2F77243046B3B4
:1006D0000CF00FCF0F77000085CF002717C03B50DD
:1006E0003195C31BD0400881033CE9F00B34D9F0AD
:1006F00020917E001981110F1213EFCF4A81441F00
:10070000093631F10D3211F0013E39F700938600C0
:100710000F903F914F911F910F912F91DF91CF91AA
:10072000CFBFCF91189520918600222389F3109195
:100730008400112369F534306AF1309384002093EA
:100740007F00109180003BE0311B3093800022C07D
:10075000009184000130E4F40AE54F7049F43091CF
:10076000600034FD18C000936000C7E6D0E017C0F9
:100770003091720034FD0FC000937200C3E7D0E0E7
:100780000EC0279598F4415099F4220F0000F9CF3C
:100790003AE501C032ED032EC0E0D0E032E017B3FD
:1007A0001660C29A17BB08B320E416E0012746E0A2
:1007B00008BB279520F4415021F4220FF9CF0127DF
:1007C00046E0000000003B5A08BBD8F2279528F409
:1007D000415029F4220F0000F9CF012746E0279568
:1007E00008BB20F4415021F4220FF9CF012746E045
:1007F00029910000332308BB21F6097F1091850061
:10080000110FC250D04008BB11F010937E0004605D
:1008100017B3197F402F497FC895C89508BB17BBF0
:1008200048BB76CF982F80916400882329F4909359
:1008300066008BB3837F8BBB9093650090936400BD
:100840000895F92FE82F80818076803279F48181B4
:10085000813061F48381813049F483E690E09093A4
:1008600083008093820081E090E0089580E090E032
:10087000089594B714BE8FEC81BF80E888B988E1F1
:1008800081BD11BC93FF0AC086B3867039F080E445
:100890008BBF80E385BF78948895F89480E285BF0C
:1008A0008BE080B983E083BF88E081BD87EF8BBB9D
:1008B0008CE08ABB89E088BB5DDC789410E000E0C6
:1008C00001C01F2DF09081008895A8955DDCF11680
:1008D000C9F3209164002223C9F0909166008091B1
:1008E0006300882311F038E001C034E0915029F40E
:1008F0008BB383278BBB90916500215019F48BB388
:10090000832B8BBB209364009093660080917200D0
:1009100084FF07C0002339F061E083E690E060DDEA
:1009200002C0002371F609B3809163000095037043
:10093000082709F4C6CF802780936300882319F025
:0E094000DB9ADA98BECFDA9ADB98BBCFFFCFF6
:02094E005AFF4E
:00000001FF
